:020000040800F2
:10000000780600207D0D00082D0300082F0300084E
:1000100033030008370300083B030008000000001A
:100020000000000000000000000000003F03000886
:1000300041030008000000004303000845030008D6
:10004000970D0008970D0008970D0008970D000800
:10005000970D0008970D0008970D0008970D0008F0
:10006000970D0008970D0008970D0008970D0008E0
:10007000970D0008970D0008970D0008970D0008D0
:10008000970D0008970D0008970D0008970D0008C0
:10009000970D0008970D0008970D0008970D0008B0
:1000A000970D0008970D0008970D0008970D0008A0
:1000B000450B0008970D0008970D0008970D0008E4
:1000C000970D0008970D0008970D0008970D000880
:1000D000970D0008970D0008A3060008970D00086B
:1000E000970D0008970D0008970D0008DFF80CD059
:1000F00002F08AFD00480047010100087806002050
:1001000086B001260027002500F06EFD4FF4A060A8
:1001100000F046FE4FF4E13000F0DFFD41F61F41F4
:1001200041F2873000F0E0FC00F0FEF94FF47A7005
:1001300000F097FD00F033FACCE0012F71D10020E0
:100140006549086065480078012816D17EB9644881
:10015000028864A101A802F007FE01A802F04DFB8D
:10016000C4B2214601A800F0B0FB064602E000F050
:10017000CCFB06460020594908700A2000F0E5FB38
:100180000546002DD8D05BA1284602F01AFB18B115
:100190000020594908609DE058A1284602F011FB53
:1001A00018B101205449086094E055A1284602F096
:1001B00008FB20B100205049091F08608AE051A1C6
:1001C000284602F0FEFA20B101204B49091F0860C1
:1001D00080E04DA1284602F0F4FA20B10020464903
:1001E0000839086076E049A1284602F0EAFA20B111
:1001F00001204149083908606CE045A1284602F019
:10020000E0FA20B100203C490C39086062E041A1CD
:10021000284602F0D6FA28B1012037490C39086087
:1002200058E050E03CA1284602F0CBFA60B1012032
:10023000314908603949C1F89C012F4908390860E3
:100240003649C1F8940145E035A1284602F0B9FAD3
:1002500060B10020284908603049C1F89C01264956
:10026000083908602D49C1F8940133E02DA12846D2
:1002700002F0A7FA30B300245421284602F0B3FA62
:100280000446641CA0783A281CD161782078303864
:1002900000EB800001EB40003038C0EB0010810023
:1002A000E078303800EB800001EB40002179084411
:1002B00030380B49088008460088002802DD0120FC
:1002C0001949087006E001200349086000F074FA3B
:1002D00000B9012731E70000B40122425400002098
:1002E0005600002048656172744F4B2020256864D9
:1002F0000D0A000051310000A08121424731000069
:1003000051320000473200005133000047330000F3
:1003100051340000473400004F464600008021421F
:100320004F4E00005400000055000020704700BFF1
:10033000FEE700BFFEE700BFFEE700BFFEE7704735
:1003400070477047704700000CB500200190009086
:100350006C48006840F480306A49086000BF694812
:10036000006800F4003000900198401C0190009853
:1003700018B90198B0F5A06FF1D16248006800F497
:10038000003010B10120009001E0002000900098A2
:10039000012843D15C48006840F010005A490860C9
:1003A0000846006820F0030008600846006840F036
:1003B0000200086053484068524948600846406857
:1003C00048600846406840F48060486008464068DD
:1003D00020F47C1048600846406840F4E81048600B
:1003E0000846006840F08070086000BF454800681B
:1003F00000F000700028F9D04248406820F0030067
:10040000404948600846406840F00200486000BF2C
:100410003C48406800F00C000828F9D10CBD10B52C
:10042000FFF792FF10BD10B53648006840F001009C
:1004300034490860084640683449084031494860FA
:1004400008460068324908402E490860084600689E
:1004500020F4802008600846406820F4FE004860D0
:100460004FF41F008860FFF7DAFF4FF00060294962
:10047000086010BD10B5002100200022214B5B68F0
:1004800003F00C0121B1042906D0082928D107E086
:10049000214B224C236027E01F4B204C236023E09C
:1004A000184B5B6803F47010164B5B6803F48032E2
:1004B000022303EB904022B9194B4343174C2360AE
:1004C0000DE0104B5B6803F4003323B1144B43433E
:1004D000124C236003E0104B4343104C236003E0B5
:1004E0000D4B0E4C236000BF00BF064B5B68C3F38F
:1004F00003130C4CE15C094B1B68CB40074C236099
:1005000010BD000000100240002002400000FFF873
:10051000FFFFF6FE08ED00E000127A000000002068
:1005200000093D000400002008B50121182000F05A
:10053000C1FF4FF40050ADF8000010208DF803000B
:1005400003208DF8020069460D4800F0F7FC4FF4D7
:1005500000510B4800F09FFD4FF4F070ADF8000023
:1005600010208DF8030003208DF80200694605482D
:1005700000F0E4FC4FF4F071024800F08CFD08BD7F
:1005800000100140000C014010B500208749088090
:100590004FF4FA718548001D02F008F910BD00B54E
:1005A00087B00121042000F085FF0121480400F0FC
:1005B0008EFF18208DF81B000420ADF818000320D2
:1005C0008DF81A0006A97A4800F0B8FC04208DF8CE
:1005D0001B000820ADF8180003208DF81A0006A9AA
:1005E000734800F0ABFC4FF4E13002900020ADF80E
:1005F00014000C20ADF812000020ADF81000ADF88A
:100600000E00ADF80C0002A96A4800F0FAFF0121C3
:10061000684801F082F8012240F22551654801F056
:1006200088F826208DF8040001208DF807008DF849
:1006300005008DF8060001A800F0B7FBFFF7A4FF46
:1006400007B000BD70B504460D46002611E04021FC
:10065000584801F04AF914F8011B564801F0CAF84D
:1006600000BF4021534801F033F90028F9D0701C35
:1006700086B2AE42EBDB70BD4C48008808B9012061
:1006800070474A48008849494988884203D1002078
:1006900046490880F4E745480088444948800120DD
:1006A000EEE710B540F22551424801F027F9B8B104
:1006B0003E480088B0F5FA7F02D300203B4908800D
:1006C0003C48001D0088C1B2384802880088401CA0
:1006D000364B1880181D81542021364801F005F949
:1006E00010BD2DE9F04105460E461446284602F09D
:1006F00084F887B239462846FFF7A4FF10E0FFF7D9
:10070000BBFF50B931462948001D02F05AF820B10C
:10071000FFF73AFF0020BDE8F0810A2000F0A1FABF
:100720002000A4F10104EAD10120F4E70FB430B5B0
:10073000CBB0054601AC50A8009001A8009A4F9993
:1007400002F026FB002000900BE014F8011B284665
:1007500001F050F800BF4021284601F0B9F8002808
:10076000F9D020780028F0D14BB030BC5DF814FBF4
:100770002DE9F04107460C461546002611E04021C0
:100780000C4801F0B2F814F8011B384601F032F8B9
:1007900000BF4021384601F09BF80028F9D0701CBA
:1007A00086B2AE42EBDBBDE8F08100007C000020A9
:1007B000000801400044004010B5754890F83C0026
:1007C000C0F38300062874D2DFE800F0031A2B4040
:1007D0005162FFF7D9FE08216EA0FFF733FF962084
:1007E00000F03FFA6E496FA002F0AEFAFFF7CCFEC0
:1007F0006748808F20F03C00001D6549888758E0DD
:1008000078A002F0A1FA32227AA17BA0FFF769FF5B
:1008100030B95F48808F20F03C0008305C49888701
:1008200047E077A002F090FA322272A179A0FFF798
:1008300058FF30B95648808F20F03C000C305449A6
:1008400088874FF4FA7000F00CFA32E074A002F0DE
:100850007BFA322267A178A0FFF743FF30B94C48FA
:10086000808F20F03C0010304949888721E076A035
:1008700002F06AFA32225FA179A0FFF732FF30B9A5
:100880004348808F20F03C0014304149888710E0B5
:1008900077A002F059FA322256A17DA0FFF721FF7E
:1008A00030B93B48808F20F03C00183038498887A9
:1008B00000BF00BF364890F83C00C0F38300062814
:1008C00001D1002010BD0120FCE730B58BB00546FA
:1008D0000C46282101A801F069FF224672A101A857
:1008E00002F042FA322275A101A8FFF7FAFE10B118
:1008F00001200BB030BD322271A12846FFF7F1FE76
:1009000008B10120F5E70020F3E770B50025642465
:100910000E216DA0FFF796FE0EE0FFF7ADFE40B989
:100920006DA11F4801F04DFF08B1002500E003252F
:1009300006E0022000F095F9601EC0B20400ECD180
:1009400000BF04B90225284670BD70B505460024D5
:1009500000BFFFF791FE80B962A1114801F031FF9D
:10096000044654B13A21204601F03DFF044614B13B
:10097000641C204670BD0020FCE7052000F071F9E2
:100980002800A5F101018DB2E3D100BFF2E700001C
:100990001400002041542B474D520D0A0000000066
:1009A000800000200D0A2A2A2A2A2A2A2A2A2A2AEC
:1009B0002A2A2A2A2A2A2A2A2A2A2A2A2A2A2A2A97
:1009C0000D0A25730D0A2A2A2A2A2A2A2A2A2A2ABD
:1009D0002A2A2A2A2A2A2A2A2A2A2A2A2A2A2A2A77
:1009E0000D0A0000415020546970733A0941540DBA
:1009F0000A0000004F4B000041540D0A00000000A7
:100A0000415020546970733A0941542B5253540D8C
:100A10000A00000041542B5253540D0A00000000FC
:100A2000415020546970733A0941542B43574D4F3C
:100A300044453D320D0A000041542B43574D4F446D
:100A4000453D320D0A000000415020546970733A50
:100A50000941542B4349504D55583D310D0A000072
:100A600041542B4349504D55583D310D0A0000006B
:100A7000415020546970733A0941542B43495053F3
:100A800045525645523D312C3838380D0A00000089
:100A900041542B4349505345525645523D312C3811
:100AA00038380D0A0000000041542B43495053458B
:100AB0004E443D302C25640D0A0000003E0000002D
:100AC00053454E44204F4B0041542B4349505354FF
:100AD000415455530D0A00002B434950535441547F
:100AE00055533A00495044007FB505460C46012154
:100AF000084600F0ECFCADF80850ADF804400020CA
:100B0000ADF80A00ADF8060001A94FF0804001F0F1
:100B10000DF801221146900701F07FFB1C208DF893
:100B2000000001208DF8010003208DF80200012053
:100B30008DF80300684600F038F90121880701F0BC
:100B400051FB7FBD10B50121880701F014FE00287C
:100B50003BD00121880701F01FFE1C480068401CA3
:100B60001A490860084600680A2804D30020086073
:100B700001201749087017480078012825D1164828
:100B80000078401C144908700846007802281CDBD5
:100B90000020087011480088002804DD0F480088F4
:100BA000401E0E4908800D48008870B90020094990
:100BB000087001200A4908600A49C1F89C010849E7
:100BC000083908600749C1F8940110BD5C00002095
:100BD000540000205500002058000020560000203E
:100BE000A08121420080214210B56FF0040000F086
:100BF00026F92E4800682E49B0FBF1F02D49087007
:100C00000846007800EB4001C1EBC0104FF6FF71C1
:100C100001EAC0002849088010BD0146254A127823
:100C20004A434FF0E0235A6100229A611A46126942
:100C300042F001021A6100BF4FF0E022106900F09B
:100C400001021AB100F48032002AF5D04FF0E02200
:100C5000126922F001024FF0E0231A6100229A612A
:100C600070470146144A12884A434FF0E0235A6104
:100C700000229A611A46126942F001021A6100BF0D
:100C80004FF0E022106900F001021AB100F4803246
:100C9000002AF5D04FF0E022126922F001024FF055
:100CA000E0231A6100229A617047000000000020D2
:100CB00000127A006000002062000020014600BFA0
:100CC000704700BF2B4A128802F04002002AF9D078
:100CD000C2B2284B1B1D1A80704710B586B004465F
:100CE000012144F2040000F0E5FB4FF40070ADF880
:100CF000140003208DF8160018208DF8170005A9A0
:100D00001D4800F01BF94FF48060ADF8140004207A
:100D10008DF8170005A9184800F010F925208DF866
:100D2000000002208DF8010003208DF80200012050
:100D30008DF80300684600F038F801940020ADF803
:100D40000800ADF80A00ADF80C00ADF810000C205A
:100D5000ADF80E0001A9074800F053FC012240F253
:100D60002551044800F0E5FC0121024800F0D5FCC3
:100D700006B010BD00380140000801400648804719
:100D800006480047FEE7FEE7FEE7FEE7FEE7FEE770
:100D9000FEE7FEE7FEE7FEE727040008ED00000897
:100DA00031490143314A1160704770B50021002379
:100DB0000F22C47804B32D4C246804F4E064C4F515
:100DC000E064210AC1F10403CA40447804FA03F143
:100DD0008478144021430901254C0678A1550478F4
:100DE00004F01F050124AC4005786D11AD0005F13C
:100DF000E025C5F8004109E0047804F01F0501244E
:100E0000AC401C4D0678761145F8264070BD1A4A54
:100E10000A400243154B1B1F1A60704739B1134A31
:100E2000121D12680243114B1B1D1A6006E00F4A87
:100E3000121D126882430D4B1B1D1A607047042857
:100E400008D14FF0E021096941F004014FF0E022A0
:100E5000116107E04FF0E021096921F004014FF032
:100E6000E0221161704700000000FA050CED00E07F
:100E700000E400E080E100E080FFFF1F10B50446C1
:100E8000CC48844208D10121042000F02DFB002130
:100E9000042000F029FB46E0C748844208D1012124
:100EA000082000F021FB0021082000F01DFB3AE0A3
:100EB000C248844208D10121102000F015FB002116
:100EC000102000F011FB2EE0BD48844208D1012122
:100ED000202000F009FB0021202000F005FB22E08B
:100EE000B848844208D10121402000F0FDFA0021D9
:100EF000402000F0F9FA16E0B348844208D10121FD
:100F0000802000F0F1FA0021802000F0EDFA0AE0E4
:100F1000AE48844207D10121801500F0E5FA002196
:100F2000A01500F0E1FA10BD10B50121084600F04F
:100F3000DBFA0021012000F0D7FA10BD2DE9F041C5
:100F4000024600250026002000230024002791F8F7
:100F500003C00CF00F0591F803C00CF0100CBCF1AD
:100F6000000F03D091F802C04CEA050591F800C0CB
:100F7000BCF1000F31D0146800202BE04FF0010CC1
:100F80000CFA00F3B1F800C00CEA03069E4220D12F
:100F900083004FF00F0C0CFA03F7BC4305FA03FC77
:100FA0004CEA040491F803C0BCF1280F06D14FF0BD
:100FB000010C0CFA00FCC2F814C00AE091F803C05E
:100FC000BCF1480F05D14FF0010C0CFA00FCC2F83F
:100FD00010C0401C0828D1D31460B1F800C0BCF187
:100FE000FF0F34DD546800202EE000F1080C4FF0B4
:100FF000010808FA0CF3B1F800C00CEA03069E429F
:1010000021D183004FF00F0C0CFA03F7BC4305FA13
:1010100003FC4CEA040491F803C0BCF1280F05D18D
:1010200000F1080C08FA0CF8C2F8148091F803C01B
:10103000BCF1480F07D100F1080C4FF0010808FA85
:101040000CF8C2F81080401C0828CED35460BDE8CC
:10105000F0814FF6FF710180022181700421C1707F
:1010600070470246002093680B400BB1012000E05E
:10107000002070470146886880B270470246002011
:10108000D3680B400BB1012000E0002070470146FF
:10109000C86880B2704701617047416170470AB10A
:1010A000016100E041617047C16070474FF48032D8
:1010B0000A43826181618261826982697047024666
:1010C0000020434B18684FF68073184040EA021026
:1010D00008433F4B186070473E49C8617047F0B500
:1010E0000A46002300240021002500F00046B6F146
:1010F000004F02D1364EF16901E0354E7168C0F300
:10110000034583B200F44016B6F5401F08D121F024
:1011100070612F4E766826F070662D4F7E6012E06B
:1011200000F48016B6F5801F06D1032606FA05F4F2
:10113000A14341F0706106E0460D360103FA06F660
:10114000B14341F0706122B1460D360103FA06F653
:10115000314300F00046B6F1004F02D11C4EF16160
:1011600001E01B4E7160F0BD30B500228B071C0FF3
:101170000F2303FA04F2164B08338C1053F8243073
:101180009343134C08348D1044F8253023468C10BB
:1011900053F824308C07240F00FA04F423430C4C3A
:1011A00008348D1044F8253030BD0A49DC31086020
:1011B0007047000000080140000C01400010014091
:1011C0000014014000180140001C014000200140B3
:1011D0000000014000002042DF48006840F00100AC
:1011E000DD49086008464068DC490840DA49486043
:1011F00008460068DA490840D74908600846006890
:1012000020F4802008600846406820F4FE00486012
:101210004FF41F0088607047CF49096821F480317E
:10122000CD4A11601146096821F480211160B0F5A2
:10123000803F03D0B0F5802F0ED106E0C649096883
:1012400041F48031C44A116007E0C349096841F4A0
:10125000A021C14A116000E000BF00BF704710B577
:1012600001460022002300204A11012A02D1BA4C73
:10127000236806E0022A02D1B74C236A01E0B64C8B
:10128000636A01F01F02012494401C400CB101204C
:1012900000E0002010BD38B500200090002400259B
:1012A00000BF3120FFF7DBFF05460098401C00908F
:1012B0000098B0F5A06F01D0002DF2D03120FFF7DB
:1012C000CEFF08B1012400E00024204638BD0146CD
:1012D0000020A14A106820F0F80040EAC100106028
:1012E0007047A04908607047024600209A4B586832
:1012F00020F47C1042EA01031843974B5860704772
:1013000098490866704701460020934A506820F0CB
:1013100003000843506070478F48406800F00C009D
:101320007047014600208C4A506820F0F0000843C6
:101330005060704701460020874A506820F4E06002
:1013400008435060704701460020834A506820F4EB
:10135000605040EAC1005060704729B17E4A527A1D
:1013600002437D4B5A7204E07B4A527A82437A4BA5
:101370005A7270477B49D831086070470146002097
:10138000754A506820F4404008435060704700217F
:10139000714A20321170704A82F82010012802D060
:1013A00004280AD104E001216B4A2032117005E0C3
:1013B0000521694A2032117000E000BF00BF70476C
:1013C0006949086070476449096A0143624A1162C9
:1013D0007047654944390860704730B500210022E4
:1013E000002400235C4D6D6805F00C0121B1042937
:1013F00005D0082923D105E05C4D056022E05B4D56
:1014000005601FE0544D6D6805F47012524D6D6813
:1014100005F48034022505EB92421CB9544D554326
:1014200005600BE04C4D6D6805F400351DB1504D65
:101430005543056002E04D4D5543056002E04B4DBC
:10144000056000BF00BF444D6D6805F0F00109095B
:10145000484D6B5C0568DD4045603F4D6D6805F4A7
:10146000E061090A434D6B5C4568DD4085603A4D9B
:101470006D6805F46051C90A3E4D6B5C4568DD40FE
:10148000C560354D6D6805F44041890B3A4D6B5C84
:10149000C568B5FBF3F5056130BD29B12E4A526927
:1014A00002432D4B5A6104E02B4A526982432A4B76
:1014B0005A61704729B1284A92690243264B9A61C2
:1014C00004E0254A92698243234B9A61704729B10F
:1014D000214AD2690243204BDA6104E01E4AD269F4
:1014E00082431D4BDA61704729B11B4AD26802431F
:1014F000194BDA6004E0184AD2688243164BDA606E
:10150000704729B1144A12690243134B1A6104E06F
:10151000114A12698243104B1A61704712494039CF
:10152000086070470F49C86470470B49C87170471D
:101530000948406A40F08070074948627047014698
:101540000020054A92680A400AB1012000E000200C
:101550007047014988727047001002400000FFF890
:10156000FFFFF6FE000042428004424200127A0071
:1015700000093D00680000207800002010B50446F6
:10158000FB48844209D101218803FFF7ADFF002108
:101590004FF48040FFF7A8FF32E0F648844209D1BB
:1015A00001214804FFF7ADFF00214FF40030FFF7A1
:1015B000A8FF25E0F048844209D101218804FFF703
:1015C000A0FF00214FF48020FFF79BFF18E0EB48BD
:1015D000844209D10121C804FFF793FF00214FF491
:1015E0000020FFF78EFF0BE0E548844208D101217F
:1015F0000805FFF786FF00214FF48010FFF781FFF9
:1016000010BD2DE9F04786B005460E460024A246DF
:1016100000BFA1460027B08900B100BF2F462C8A29
:101620004CF6FF700440F08804432C82AC894EF6DF
:10163000F3100440B088318908437189084304439A
:10164000AC81AC8A4FF6FF400440B0890443AC82C1
:1016500001A8FFF7C2FEC648874202D1DDF810A0FC
:1016600001E0DDF80CA0A88900F4004040B10AEBCD
:10167000CA0000EB0A1031684900B0FBF1F807E03E
:101680000AEBCA0000EB0A1031688900B0FBF1F8E0
:101690006420B8FBF0F004012009642101FB1089EB
:1016A000A88900F4004040B1322000EBC900B0FB33
:1016B000F1F000F00700044308E0322000EB0910CD
:1016C0006421B0FBF1F000F00F0004432C8106B060
:1016D000BDE8F0874FF41651016000218180C18080
:1016E00001810C21418100218181704710B50246A2
:1016F0000020108A4FF2FF0318400B884C882343C8
:101700008C882343CC8823431843108210BD0021CA
:10171000018041808180C180704721B1828942F47B
:101720000052828104E082894DF6FF731A40828163
:101730007047F0B50346002400260025002040F63F
:101740006A17B94200D100BF1846C1F3421401F034
:101750001F06012707FA06F5012C01D10C3004E021
:10176000022C01D1103000E014301AB107682F4369
:10177000076002E00768AF430760F0BD1AB1838AD3
:101780000B43838202E0838A8B4383827047028A01
:101790004FF6F0731A400282028A0A4302827047AF
:1017A00082894FF2FF731A40828182890A438281C3
:1017B000704721B1828942F00202828104E082896D
:1017C0004FF6FD731A4082817047028A4FF6DF732D
:1017D0001A400282028A0A430282704721B1028AB9
:1017E00042F48042028204E0028A4BF6FF731A4000
:1017F00002827047C1F308028280704701468888E0
:10180000C0F308007047818941F001018181704770
:10181000028BD2B20283028B42EA0122028370471A
:10182000028B02F47F420283028B0A4302837047D9
:1018300021B1828A42F02002828204E0828A4FF63D
:10184000DF731A408282704721B1828A42F010020F
:10185000828204E0828A4FF6EF731A4082827047D8
:1018600021B1828A42F00802828204E0828A4FF625
:10187000F7731A408282704721B1828942F4004294
:10188000828103E08289C2F30E028281704721B116
:10189000828A42F40062828204E0828A4FF2FF73FD
:1018A0001A4082827047828A4FF6FB731A40828206
:1018B000828A0A438282704721B1828A42F0020200
:1018C000828204E0828A4FF6FD731A40828270475A
:1018D00002460020B1F5007F00D100BF13880B4005
:1018E0000BB1012000E00020704701F40072B2F556
:1018F000007F00D100BFCA430280704770B5024626
:10190000002400230025002040F66A16B14200D1D1
:1019100000BFC1F3421501F01F03012606FA03F3CD
:10192000012D02D19689334006E0022D02D1168A9C
:10193000334001E0968A33400C12012606FA04F483
:101940001688344013B10CB1012000E0002070BDB6
:1019500010B50022002340F66A14A14200D100BF56
:101960000A1201249440A3B2DC43048010BD00009D
:10197000003801400044004000480040004C004056
:101980000050004010B50446FE48844208D10121B1
:10199000C014FFF7A9FD0021E014FFF7A5FDC4E086
:1019A000B4F1804F08D101210846FFF7AAFD0021BC
:1019B0000120FFF7A6FDB8E0F348844208D10121D9
:1019C0000220FFF79EFD00210220FFF79AFDACE008
:1019D000EE48844208D101210420FFF792FD002146
:1019E0000420FFF78EFDA0E0E948844208D10121E0
:1019F0000820FFF786FD00210820FFF782FD94E014
:101A0000E448844208D101211020FFF77AFD00212B
:101A10001020FFF776FD88E0DF48844208D10121DD
:101A20002020FFF76EFD00212020FFF76AFD7CE0FB
:101A3000DA48844208D101214014FFF755FD002106
:101A40006014FFF751FD70E0D548844209D10121AF
:101A5000C804FFF749FD00214FF40020FFF744FDC3
:101A600063E0D048844209D101210805FFF73CFD1D
:101A700000214FF48010FFF737FD56E0CA4884423A
:101A800009D101214805FFF72FFD00214FF4001077
:101A9000FFF72AFD49E0C548844208D101214020D2
:101AA000FFF72FFD00214020FFF72BFD3DE0C04850
:101AB000844208D101218020FFF723FD00218020EE
:101AC000FFF71FFD31E0BB48844208D1012180159A
:101AD000FFF717FD0021A015FFF713FD25E0B6481D
:101AE000844209D101210804FFF7FEFC00214FF4D4
:101AF0008030FFF7F9FC18E0B048844209D1012199
:101B00004804FFF7F1FC00214FF40030FFF7ECFC34
:101B10000BE0AB48844208D101218804FFF7E4FCC4
:101B200000214FF48020FFF7DFFC10BD0022028867
:101B3000944B98420ED0994B98420BD0B0F1804F05
:101B400008D0914B984205D0904B984202D0904BD0
:101B5000984204D14FF68F731A404B881A438D4B2D
:101B6000984207D08C4B984204D04FF6FF431A405E
:101B7000CB881A4302808B8883850B880385814B31
:101B800098420BD0854B984208D08B4B984205D099
:101B90008A4B984202D08A4B984201D10B7A038635
:101BA00001238382704770B5002400220023058C36
:101BB0004FF6FE7635400584028C8388048B4FF601
:101BC0008F752C40B51E2C400D882C43751E2A4065
:101BD0000D892A434D882A436A4DA8420BD06F4D88
:101BE000A84208D0744DA84205D0744DA84202D036
:101BF000734DA84213D14FF6F7752A404D892A43F9
:101C00004FF6FB752A408D882A434FF6FF652B401F
:101C10004FF6FF552B408D892B43CD892B43838075
:101C20000483CD888586028470BD70B500240022AF
:101C30000023058C4FF6EF7635400584028C8388AF
:101C4000048B48F6FF752C404FF6FF452C400D885D
:101C50004FF6FF7606EA05252C434FF6DF752A403E
:101C60000D8906EA05152A434D8806EA05152A431B
:101C7000444DA84202D0494DA8421DD14FF67F7570
:101C80002A404D894FF6FF7606EA05152A434FF69E
:101C9000BF752A408D8806EA05152A434FF6FF35A1
:101CA0002B404FF2FF752B408D8906EA85052B43AB
:101CB000CD8906EA85052B4383800483CD8805877B
:101CC000028470BD70B5002400220023058C4FF6FD
:101CD000FF6635400584028C8388848B4FF68F75B0
:101CE0002C404FF6FC752C400D882C434FF6FF55C9
:101CF0002A400D894FF6FF7606EA05252A434D88CE
:101D000006EA05252A431F4DA84202D0234DA842CA
:101D10001DD14FF2FF752A404D894FF6FF7606EA36
:101D200005252A434FF6FF352A408D8806EA05250A
:101D30002A434EF6FF752B404DF6FF752B408D89DB
:101D400006EA05152B43CD8906EA05152B4383804A
:101D50008483CD888587028470BD70B500220023FE
:101D60000024058C4EF6FF7635400584038C84886C
:101D7000828B48F6FF752A404FF6FF452A400D88B2
:101D800020E00000002C014000040040000800405A
:101D9000000C0040001000400014004000340140DE
:101DA000004C014000500140005401400018004028
:101DB000001C004000200040004001400044014061
:101DC000004801404FF6FF7606EA05252A434DF606
:101DD000FF752B400D8906EA05352B434D8806EA31
:101DE00005352B43FA4DA84202D0FA4DA84208D13E
:101DF0004BF6FF752C408D894FF6FF7606EA851568
:101E00002C4384808283CD88A0F84050038470BD29
:101E1000828B4FF2FF331A408283828B4FF6FF731F
:101E200003EA01231A4382837047F0B50C46154636
:101E3000002200210026078C4EF6FF7C07EA0C07E3
:101E40000784828B018C4FF6FF7707EA043640F651
:101E5000FF473A404FF6FF7707EA05273A434FF628
:101E6000FF7707EA03373A43D94FB8420ED0D94F2C
:101E7000B8420BD0B0F1804F08D0D74FB84205D050
:101E8000D64FB84202D0D64FB84206D14DF6FF77B2
:101E9000394046F48057394305E047F6FF5739404B
:101EA00044F48057394382830184F0BD828B4FF61E
:101EB000F3731A408283828B0A4382837047F0B5A2
:101EC0000C461546002200210026078C4FF6FF6CB9
:101ED00007EA0C070784828B018C4FF6FF7707EA2D
:101EE00004264FF60C773A404FF6FF7707EA0317C0
:101EF0002F433A43B64FB8420ED0B64FB8420BD03C
:101F0000B0F1804F08D0B44FB84205D0B34FB842BB
:101F100002D0B34FB84206D14FF6FF57394046F4CE
:101F20008077394305E04FF2FF57394044F480771A
:101F3000394382830184F0BD028B4FF2FF331A4094
:101F40000283028B4FF6FF7303EA01231A430283D5
:101F50007047F0B50C461546002200210026078C7C
:101F60004FF6EF7C07EA0C070784028B018C4FF6D3
:101F7000FF7707EA041640F6FF473A404FF6FF772F
:101F800007EA03373A434FF6FF7707EA05273A4354
:101F90008F4FB8420ED08F4FB8420BD0B0F1804F68
:101FA00008D08D4FB84205D08C4FB84202D08C4F2C
:101FB000B84206D14FF6DF77394046F01007394373
:101FC00005E04FF65F77394044F01007394302834C
:101FD0000184F0BD028B4FF6F3731A400283028B2B
:101FE0000A4302837047F0B50C46154600220021D3
:101FF000068C4FF6FE773E400684028B018C4FF62E
:102000000C7632407E1C06EA03162E433243704E95
:10201000B0420ED06F4EB0420BD0B0F1804F08D01E
:102020006D4EB04205D06D4EB04202D06C4EB04203
:1020300006D14FF6FD76314044F00106314305E00C
:102040004FF6F576314044F00106314302830184B6
:10205000F0BD70B505460C465D4885420ED05D4822
:1020600085420BD0B5F1804F08D05B48854205D042
:102070005A48854202D05A48854200D100E000BF4C
:10208000208850B92389A28861882846FFF7ABFFD2
:10209000E1882846FFF79EFF25E0208804280AD122
:1020A0002389A28861882846FFF753FFE1882846E4
:1020B000FFF742FF17E0208808280AD12389A28869
:1020C00061882846FFF7FBFEE1882846FFF7EEFE11
:1020D00009E02389A28861882846FFF7A6FEE188E7
:1020E0002846FFF795FE70BD2DE9F04105460C46E8
:1020F00000260127608808B9022600E00026A08893
:10210000012801D1022700E001272088A0B92389F6
:10211000A28861882846FFF766FFE1882846FFF716
:1021200059FF23893A4631462846FFF712FFE188D6
:102130002846FFF701FF13E02389A288618828461B
:10214000FFF707FFE1882846FFF7F6FE23893A46A6
:1021500031462846FFF747FFE1882846FFF73AFF58
:10216000BDE8F0810A884B881A438B881A43CB88D4
:102170001A430B891A434B891A438B891A43A0F8D7
:10218000442070474FF6FF71818000210180C1809B
:102190004180017270470021018041808180C180AF
:1021A000018141818181C18170470021018041808D
:1021B000012181800021C1800181704700210180BF
:1021C00041808180C180018141818181704700000F
:1021D000002C014000340140000400400008004091
:1021E000000C004021B1028842F00102028004E0AC
:1021F00002884FF6FE731A400280704731B1B0F882
:10220000442042F40042A0F8442005E0B0F8442005
:10221000C2F30E02A0F8442070471AB183890B4321
:10222000838102E083898B43838170478182704779
:1022300041EA0203A0F8483070471AB183890B4382
:10224000838102E083898B438381704701894FF644
:10225000F8721140018170470A46002101894FF64A
:102260008F73194011430181704730B504460D4604
:1022700029462046FFF7F0FF208940F00700208123
:1022800030BD2DE9F04104460D4616461F46602D2F
:1022900006D13B46012231462046FFF75AFE05E0B3
:1022A0003B46012231462046FFF79DFE2946204647
:1022B000FFF7D2FF208940F007002081BDE8F081C0
:1022C00030B50C4600210189C9B24FF6FF7505EA09
:1022D0000325154325432943018130BD2DE9F041F4
:1022E00005460E4617469846002443463A46314670
:1022F0002846FFF7E5FF2C894FF6F870044044F0BC
:1023000007044FF68F70044044F070042C81BDE840
:10231000F081F0B504460D4616461F463B46324650
:1023200029462046FFF7CCFF208940F480402081D9
:10233000F0BD0185828270470A46002101884FF670
:102340008F731940114301807047F0B50C46154654
:102350001E460021002200230189028B038C4FF6C8
:10236000F877394021434FF6FC473A4040F20117D5
:102370003A434FF6DD773B404FF6FF7707EA061703
:102380002F433B43018102830384F0BD0A460021B1
:10239000018B4FF68F7319401143018370470A4632
:1023A0000021018B48F6FF7319404FF6FF7303EAD3
:1023B00002231943018370470A460021818B4FF69F
:1023C0008F7319401143818370470A460021818B26
:1023D00048F6FF7319404FF6FF7303EA02231943CF
:1023E0008183704721B1028842F08002028004E0BC
:1023F00002884FF67F731A400280704721B18288AD
:1024000042F00402828004E082884FF6FB731A4097
:102410008280704721B1828842F00802828004E005
:1024200082884FF6F7731A408280704721B1828804
:1024300042F00102828004E082884FF6FE731A4067
:10244000828070470A460021018B4FF6F7731940CE
:102450001143018370470A460021018B4FF2FF733D
:1024600019404FF6FF7303EA0223194301837047B3
:102470000A460021818B4FF6F7731940114381837F
:1024800070470A460021818B4FF2FF7319404FF6C7
:10249000FF7303EA02231943818370470A46002130
:1024A000018B4FF6FB7319401143018370470A46B5
:1024B0000021018B4FF6FF3319404FF6FF7303EAFB
:1024C00002231943018370470A460021818B4FF68E
:1024D000FB7319401143818370470A460021818BA9
:1024E0004FF6FF3319404FF6FF7303EA02231943F7
:1024F000818370470A460021018B4FF67F73194094
:102500001143018370470A460021018BC1F30E017C
:102510004FF6FF7303EA02231943018370470A460B
:102520000021818B4FF67F731940114381837047DF
:102530000A460021818BC1F30E014FF6FF7303EAB7
:1025400002231943818370470A460021018C4FF60C
:10255000FD7319401143018470470A460021018C24
:102560004FF6F77319401143018470470A46002162
:10257000018C4FF6DF7319404FF6FF7303EA021325
:102580001943018470470A460021018C4FF67F737E
:1025900019404FF6FF7303EA021319430184704791
:1025A0000A460021018C4FF6FF5319404FF6FF7386
:1025B00003EA02231943018470470A460021018C73
:1025C0004FF2FF7319404FF6FF7303EA02231943DA
:1025D000018470470A460021018C4DF6FF731940B3
:1025E0004FF6FF7303EA023319430184704730B595
:1025F000002301248C40A3B2048C9C430484048CEB
:1026000002FA01F5ADB22C43048430BD30B500238D
:1026100004248C40A3B2048C9C430484048C02FAEE
:1026200001F5ADB22C43048430BD70B503460020E3
:1026300000241846183001258D40ACB21D8CA543EE
:102640001D8409B1082909D100EB6100056825F056
:10265000700505600568154305600EE00D1FC5F3A4
:102660004E052844056825F4E045056005684FF6E9
:10267000FF7606EA02263543056070BD21B1028867
:1026800042F00202028004E002884FF6FD731A4015
:102690000280704721B1028842F00402028004E007
:1026A00002884FF6FB731A400280704721B182887E
:1026B00042F08002828004E082884FF67F731A40E5
:1026C0008280704702884FF6F7731A4002800288B2
:1026D0000A430280704782884FF68F731A408280C7
:1026E00082880A438280704702894FF6F8731A4045
:1026F000028102890A430281704702894FF67F7383
:102700001A40028102890A4302817047818470471E
:102710008185704781867047018770478187704740
:10272000A0F84010704702884FF6FF431A4002801D
:1027300002880A43028070470146888E704701462E
:10274000088F70470146888F70470146B1F84000F6
:1027500070470146888C70470146088D70470246D5
:102760000020138A0B400BB1012000E000207047CD
:10277000CA430282704730B502460020002300247D
:10278000158A05EA0103958905EA010413B10CB124
:10279000012000E0002030BDCA4302827047D2B25F
:1027A00001E000F8012B491EFBD270470022F6E73A
:1027B00010B513460A4604461946FFF7F0FF2046B7
:1027C00010BD30B505462A460B4612F8010B13F82A
:1027D000014B08B1A042F8D01CB1002802D06D1CFA
:1027E000F1E7284630BDCAB2401E10F8011F8A42E8
:1027F00002D00029F9D100207047421C10F8011BBB
:102800000029FBD1801A704730B50B4601460020E5
:102810002022012409E021FA02F59D4205D303FAA2
:1028200002F5491B04FA02F52844151EA2F1010223
:10283000F1DC30BD2DE9F05F0546002092469B4655
:1028400088460646814640241BE0284641464746C6
:10285000224600F0FAF953465A46C01A914110D365
:1028600011461846224600F0E1F92D1A67EB0108DF
:102870004F4622460120002100F0D8F917EB00094D
:102880004E41201EA4F10104DFDC484631462A46B1
:102890004346BDE8F09F2DE9FE4F804681EA0300E4
:1028A000C00F0C46009021F0004123F00045B8EB2A
:1028B0000200A94105D24046214690461C460B46DF
:1028C000024623F00040104347D0270DC7F30A000B
:1028D000C3F30A510290401A019040286BDAC3F307
:1028E000130040F4801B0098924620B10023D2EBE5
:1028F000030A63EB0B0B01985946C0F140025046A6
:1029000000F094F906460D4650465946019A00F0EB
:10291000ACF910EB08006141002487EA115284EA07
:10292000E7731A4340D0009A62B3019A012A4FEA32
:10293000075215DC001B61EB02014FF0004202EA76
:102940000752CDE90042001C41F5801132462B466A
:1029500000F0ACF903B0BDE8F08F40462146F9E73E
:10296000001B61EB0201001C41F5801300185B4164
:102970002018A2F5001747EB030140EAD570B619FD
:102980006D4111E06D084FEA360645EAC0754FEA21
:102990000752001B61EB0201001C41F58011490840
:1029A0004FEA30000019514132462B4603B0BDE8D2
:1029B000F04F00F06CB90098012240000023D0EBEA
:1029C000020263EBE073009821464FEAE074B8EB33
:1029D000000061EB0401E9E783F000435BE781F06D
:1029E000004158E72DE9FE4F81EA030404F000445A
:1029F00021F0004100944FF0000B23F0004350EA17
:102A000001045ED052EA03045BD0C3F30A54C1F35D
:102A10000A552C44A4F2F3340194A0FB0254C1F3F0
:102A2000130141F48011C3F3130343F4801301FB3A
:102A3000024400FB034E840A970A44EA815447EAA1
:102A40008357A4FB076802958D0A05FB07854FEAAB
:102A5000932C04FB0C542705029D4FEA065847EAC5
:102A60001637B5EB08056EEB070C870E920E47EA9A
:102A7000811742EA8312A7FB0201B6EB0B0164EB5C
:102A800000042B0D43EA0C335E1844EB1C50DA466D
:102A90005146E7FB0201C5F313044FEA0B3343EA47
:102AA00014534FEA0432019C43EA0603A4F10C04D8
:102AB0000294009CCDE900B400F0F8F803B0BDE842
:102AC000F08F00200146F9E72DE9F04D81EA03047B
:102AD00004F0004B21F0004514464FF0000A23F0AB
:102AE000004150EA050220D054EA01021DD0C5F38E
:102AF0000A570246C5F31303C1F31300C1F30A5684
:102B000040F4801543F48013A7EB0608101BD6464B
:102B100008F2FD3873EB050002D308F1010801E06B
:102B200092185B41B8F1000F03DA00200146BDE8BE
:102B3000F08D00204FF48011064684460EE0171BEE
:102B400073EB050705D3121B63EB050306434CEA41
:102B5000010C49084FEA300092185B4150EA010726
:102B6000EDD152EA030012D082EA040083EA0501A3
:102B7000084305D0101BAB4106D20122002306E01A
:102B800000224FF0004302E06FF0010253101AEBF5
:102B900006004CEB085110EB0A0041EB0B01BDE8BD
:102BA000F04D00F074B8C1F30A52C1F3130140F2C2
:102BB000FF3341F480119A4202DA00200146704747
:102BC00040F233439A42A2F2334202DC524200F016
:102BD0003CB800F02BB8000030B5041E71F10004C1
:102BE00004DB4FF00044404264EB0101141E73F11A
:102BF000000405DB1C464FF00043524263EB040324
:102C0000994208BF904230BD064C074D06E0E0688F
:102C100040F0010394E8070098471034AC42F6D323
:102C2000FDF768FABC390008DC390008202A04DB0B
:102C3000203A00FA02F1002070479140C2F12003CF
:102C400020FA03F3194390407047202A04DB203A0E
:102C500021FA02F00021704721FA02F3D040C2F1BC
:102C600020029140084319467047202A06DBCB1703
:102C7000203A41FA02F043EAE07306E041FA02F337
:102C8000D040C2F12002914008431946704710B568
:102C9000141E73F1000408DA401C41F1000192187F
:102CA0005B411A4301D120F0010010BD2DE9F04D28
:102CB00092469B4611B1B1FA81F202E0B0FA80F27D
:102CC00020329046FFF7B2FF04460F4640EA0A0062
:102CD00041EA0B0153465A46084313D0114653EAC2
:102CE000010019D0C8F140025046FFF7AEFF05467B
:102CF0000E46504659464246FFF798FF084305D016
:102D0000012004E020463946BDE8F08D002005434F
:102D100046EAE0762C4337430A986305E40AA0EBC1
:102D200008000022FD0A44EA47540A3002D5002078
:102D30000146E9E7010510196941DDE90845001977
:102D40006941BDE8F04DA2E70FB4054B10B503A9EA
:102D5000044A029800F0F0F810BC5DF814FB000083
:102D6000C30C0008640000200FB4084B10B504A980
:102D700002AA039800F0E0F8044602A9002000F03F
:102D800013FE204610BC5DF814FB0000A9390008B2
:102D900037B514460846064B6A46214600F044FA09
:102DA00004466946002000F004FE20463EBD0000B7
:102DB000B339000802E008C8121F08C1002AFAD17E
:102DC00070477047002001E001C1121F002AFBD1AB
:102DD000704700002DE9FF5FDDE90220010DDDF8FD
:102DE00038B0024318D044F61050A1F2FF314143ED
:102DF0000D140F98012820D0A5EB0B00401C5FEAB2
:102E0000000A4FF00004474EDFF81C91A0465046E0
:102E100016D5CAF1000728E00F98012443A2012823
:102E200008D0002100980F9BC0E90021C0E90243AF
:102E3000BDE8FF9F6FEA0B01F4E7CBF10000DEE78E
:102E4000074612E0F80707D0224633464046494677
:102E5000FFF7C8FD8046894622463346104619468C
:102E6000FFF7C0FD04460E467F10002FEAD1DDE9D2
:102E70000201BAF1000F42464B4602DAFFF7B2FDFB
:102E800001E0FFF721FE04460E460022284BFFF723
:102E9000A3FE03D84FF0FF30014607E00022254B88
:102EA00020463146FFF7F7FCFFF77DFE102409E0CE
:102EB000002C0ADB0A220023FFF7BCFC019B303206
:102EC0001A55641E50EA0102F2D1641C019AC4F141
:102ED000110314440F9A012A03D0012208430DD193
:102EE0000AE0084304D000204FF0110B0F9080E758
:102EF000A3EB0B056D1E0DE05B4504DD4FF00002FA
:102F000005F1010504E003DA4FF00002A5F1010527
:102F1000002AECD000980F99C0E90231C0E90045C1
:102F200086E70000000024400000F03F3000000071
:102F30000000F0430000E03F2DE9FF4F8BB08846D2
:102F40000546002606E025280BD0DDE90D12904746
:102F50006D1C761C28780028F5D10FB03046BDE8EE
:102F6000F08F0024A146A2460122AE4900E00443AE
:102F700015F8013F203B02FA03F00842F7D1287808
:102F80002A2810D06FF02F022878A0F130010929EB
:102F900015D809EB890102EB410144F0020400EB72
:102FA00001096D1CF0E758F8041B5FEA010903D51D
:102FB00044F40054C9F1000944F002046D1C28785F
:102FC0002E2817D115F8010F44F004042A280ED03A
:102FD0006FF02F022878A0F1300109290AD80AEBF6
:102FE0008A0102EB410100EB010A6D1CF2E758F87F
:102FF00004AB6D1C28786C280FD006DC4C2817D049
:1030000068280DD06A2814D104E0742810D07A28DA
:103010000FD10DE044F400140AE044F4801401E000
:1030200044F440146978814202D104F580146D1C87
:103030006D1C2878692865D006DC00288DD06328AF
:1030400027D0642806D15DE06E2808D073282AD0E6
:10305000752877D0DDE90D129047761CE0E0C4F3C7
:103060000250022809D003280DD0D8F800100428F7
:103070000DD00E6008F10408D2E0D8F80010F21765
:10308000C1E90062F6E7D8F800100E80F2E70E7092
:10309000F0E718F8041B8DF8001000208DF80100EF
:1030A000EB46012003E058F804BB4FF0FF30610706
:1030B0004FF0000701D40AE07F1C57450DDA874224
:1030C000FADB1BF807100029F6D106E07F1C8742C7
:1030D000FCDB1BF807100029F8D1DDE90D23A9EB73
:1030E00007008146214600F031FC3044C61904E057
:1030F000DDE90D121BF8010B90477F1EF8D2214627
:10310000484688E058F8040BC4F302514FF00A0B0C
:10311000032900D100B2042900D140B2002802DA0C
:1031200040422D2102E0210505D52B218DF82410E8
:10313000012104E006E0E10710D02021F6E708AF06
:10314000089113E058F8040BC4F302514FF00A0B36
:10315000032900D180B2042900D1C0B20021EEE7DA
:103160005946FFF751FB303107F8011D0028F7D110
:10317000ADEB070000F1200B600702D524F480348A
:1031800001E04FF0010ADA4502DDAAEB0B0000E096
:103190000020824600EB0B0108980144A9EB0100D6
:1031A0000A90E00306D4DDE90D2321460A9800F0D9
:1031B000CDFB06444FF0000908E009A911F8090009
:1031C000DDE90D12904709F10109761C089989453E
:1031D000F3DBE0030CD5DDE90D2321460A9800F06E
:1031E000B5FB064404E0DDE90D1230209047761C63
:1031F000BAF10001AAF1010AF5DC05E0DDE90D12E2
:1032000017F8010B9047761CBBF10001ABF1010BE5
:10321000F4DC0A982146DDE90D2300F073FB064437
:103220006D1C97E6092801002DE9FF4F95B09B46DC
:103230008946064600250FE2252877D10024274637
:10324000F84A0121059400E0044316F8013F203BB1
:1032500001FA03F01042F7D130782A2811D06FF02C
:103260002F033078A0F13002092A16D8059A44F0CD
:10327000020402EB820203EB42021044761C05902A
:10328000EFE759F8042B0592002A03DA504244F480
:103290000054059044F00204761C30782E2816D194
:1032A00016F8010F44F004042A280DD06FF02F0205
:1032B0003078A0F13003092B09D807EB870302EB24
:1032C0004303C718761CF3E759F8047B761C307863
:1032D0006C280FD006DC4C2817D068280DD06A283F
:1032E00014D104E0742810D07A280FD10DE044F4F2
:1032F00000140AE044F4801401E044F440147278AD
:10330000824202D104F58014761C761C307866283F
:103310000BD013DC582877D009DC002875D045285D
:10332000F6D04628F4D047281AD19DE118E063284A
:1033300035D0642879D0652812D195E1702873D0F2
:1033400008DC6728F1D069286FD06E280DD06F286F
:1033500006D1B5E073282CD0752875D0782874D0A4
:103360005A46179990476D1C75E1C4F30250022824
:1033700009D003280DD0D9F8001004280DD00D6015
:1033800009F1040967E1D9F80010EA17C1E9005210
:10339000F6E7D9F800100D80F2E70D70F0E719F8A4
:1033A000041B8DF8001000208DF80100EA46012072
:1033B00003E059F804AB4FF0FF3061074FF0000114
:1033C00002D40DE008F101018846B9420FDA8045C8
:1033D000F8DB1AF808100029F4D108E008F101011F
:1033E00088468142FADB1AF808100029F6D10598C0
:1033F0005B46A0EB080721463846179A00F0BDFA55
:10340000284400EB080507E04DE029E10DE01AF83B
:10341000010B5A4617999047B8F10108F7D25B465D
:1034200021463846179A13E142E00A220092C4F37B
:1034300002524FF0000A022A08D059F804CB032A9E
:103440004FEAEC710AD00DE029E02AE009F107010A
:1034500021F00702F2E802C1914609E00FFA8CFC64
:103460004FEAEC71042A03D14FFA8CFC4FEAEC715D
:10347000002907DA0A460021DCF1000C61EB0201A9
:103480002D2202E0220504D52B228DF804200122F2
:1034900003E0E20701D02022F7E7904659E00A2135
:1034A00002E010220DE010214FF0000A00910BE025
:1034B00010224FF0000A44F004040827009203E0B1
:1034C00008224FF0000A0092C4F30252022A05D0EB
:1034D00059F804CB0021032A08D009E009F10701BB
:1034E00021F00702F2E802C1914605E01FFA8CFCC8
:1034F000042A01D10CF0FF0C4FF00008220728D558
:10350000702806D0009B83F0100353EA0A0305D00D
:103510000EE040228DF80420012208E05CEA01025E
:1035200006D030228DF804208DF805000222904646
:10353000009B83F0080353EA0A030AD15CEA010204
:1035400001D1620705D530228DF804204FF0010823
:103550007F1E582804D034A003900EA802900DE0DE
:1035600036A0F9E753466046009AFFF763F98446B0
:103570000398825C0298401E029002705CEA01008F
:10358000F0D1029806A9081A00F1200A600702D5B6
:1035900024F4803400E00127574502DDA7EB0A0040
:1035A00000E0002000EB0A01009005984144401A19
:1035B0000590E00306D45B462146179A059800F073
:1035C000DCF90544002706E001A85A46C05D1799BA
:1035D00090476D1C7F1C4745F6DBE0030CD55B462E
:1035E0002146179A059800F0C8F9054404E03020F8
:1035F0005A46179990476D1C0099481E0090002963
:10360000F5DC08E0029802995A460078491C0291BC
:10361000179990476D1CBAF10001AAF1010AF1DC7B
:1036200065E1000009280100303132333435363786
:1036300038396162636465660000000030313233FE
:10364000343536373839414243444546000000009E
:1036500000F06AF90544761C307800287FF4ECAD60
:1036600019B02846BDE8F08F620700D4062709F19B
:10367000070222F0070CFCE80223E14603F00048B1
:103680005FEA080C02D00FF2702C0DE05FEA045CD8
:1036900002D50FF2682C07E05FEAC47C02D00FF27B
:1036A000602C01E0AFF2700C4FF0FF3823F00043C4
:1036B000CDF850C065280CD006DC452809D0462836
:1036C0001DD047283DD13DE0662818D067287ED11F
:1036D00038E00021112F01DB112000E0781CCDE93A
:1036E000000106A90EA8FFF775FBDDE90F010E9A90
:1036F00003910021009207F1010A04914DE04FF07F
:1037000000400097CDE9011006A90EA8FFF762FB63
:10371000DDE90F0203920E9B11990022DDF80CA047
:103720000093049211B9791C00EB010AB7EB0A006F
:1037300004D4C0F1FF3007F1010A0490AAEB07009E
:10374000019044E0012F00DA01270021112F01DD53
:10375000112000E03846CDE9000106A90EA8FFF7C8
:1037600039FBDDE90F010E9A0391002104910092CB
:10377000BA4621070CD40399514500DA8A46BAF1BA
:10378000010F05DD009AAAF10101515C302908D032
:10379000B84202DA10F1040F06DA0121CDE9011076
:1037A00015E0AAF10101E9E7002805DC04990144CC
:1037B0000491AAEB000102E0411C514500DD8A465C
:1037C0000499401A401C01904FF0004002902007DD
:1037D00004D40198504501DBCDF8048000208DF819
:1037E0004F0002980DF14F07B0F1004F25D02B206C
:1037F0000E9002984FF0020800280CDA4042029026
:103800002D200E9007E00A210298FEF7FDFF3031CF
:10381000029007F8011DB8F10001A8F10108F2DCDF
:1038200002980028EFD1791E0E980870307800F0C9
:10383000200040F0450007F8020D12A8C01B00F15F
:1038400007081498007800B1012000EB0A010198E4
:1038500001EBE07105984144401A401E0590E003D9
:1038600006D45B462146179A059800F086F8054471
:103870001498007818B15A46179990476D1CE003C8
:1038800024D55B462146179A059800F076F8054442
:103890001CE00498002807DBDDE90301884203DD12
:1038A0000098405C179901E0179930205A469047DC
:1038B000049805F10105401C04900198401E0190F8
:1038C00004D12E205A46179990476D1CBAF1000179
:1038D000AAF1010ADDDC05E017F8010B5A46179939
:1038E00090476D1CB8F10001A8F10108F4DC5B46BB
:1038F0002146179A0598ABE62D0000002B0000002A
:10390000200000002DE9F041044600251E46174620
:10391000880404D405E039462020B0476D1C641E9D
:10392000F9D52846BDE8F0812DE9F041044600258F
:103930001E461746880404D405E039462020B047C7
:103940006D1C641EF9D52846BDE8F0812DE9F041D3
:10395000044600251E469046C80301D5302700E0E6
:103960002027880404D505E041463846B0476D1C41
:10397000641EF9D52846BDE8F0812DE9F0410446E2
:1039800000251E469046C80301D5302700E02027B9
:10399000880404D505E041463846B0476D1C641ED6
:1039A000F9D52846BDE8F0810A68531C0B601070F9
:1039B00070470A68531C0B6010707047DC390008B0
:1039C000000000207C000000B42D0008583A0008D8
:1039D0007C000020FC050000C42D000800A24A0461
:1039E00000000000000000000102030406070809AF
:1039F00000000000000000000000000000000000C7
:103A000000000000000000000000000000000000B6
:103A100000000000000000000000000000000000A6
:103A20000000000000000000000000000001000095
:103A30000100000000000000000000000000000085
:103A40000000000000000000010203040102030462
:083A500006070809020406083C
:04000005080000ED02
:00000001FF
